:020000040800F2
:1000000000040024A10200088D0E0008910E0008D3
:10001000E10E0008910E0008B90E0008A3020008C6
:10002000A3020008A3020008A30200084925000853
:10003000A3020008A3020008A3020008A30200080C
:10004000A3020008A3020008A3020008A3020008FC
:10005000A3020008A3020008813A0008AD3A000894
:10006000D93A0008053B0008313B0008A30200080C
:10007000A3020008A3020008A3020008A3020008CC
:10008000A3020008A3020008A3020008A3020008BC
:10009000A3020008A3020008A30200085D3B0008B9
:1000A000A3020008A3020008A3020008A30200089C
:1000B000FD360008A3020008A3020008A3020008FE
:1000C000A3020008A3020008A3020008A30200087C
:1000D000A3020008A3020008A3020008A30200086C
:1000E000C53B0008A3020008A3020008A302000801
:1000F000A3020008A3020008A3020008A30200084C
:10010000A3020008A3020008A3020008A30200083B
:10011000A3020008A3020008A3020008A30200082B
:10012000A3020008A3020008A3020008A30200081B
:10013000A3020008A3020008A3020008A30200080B
:10014000A3020008A3020008A3020008A3020008FB
:10015000A3020008A3020008A3020008A3020008EB
:10016000A3020008A3020008A3020008A3020008DB
:10017000A302000881300008A3020008A3020008BF
:10018000A3020008A3020008310F0008A302000820
:10019000A3020008A3020008A3020008A3020008AB
:1001A000A3020008A3020008A3020008A30200089B
:1001B000A3020008A3020008A3020008A30200088B
:1001C000A3020008A3020008A3020008A30200087B
:1001D000A30200086D300008A3020008A302000873
:1001E000A3020008A3020008A3020008A30200085B
:1001F000A3020008A3020008A3020008A30200084B
:10020000A3020008A3020008A3020008A30200083A
:10021000A3020008A3020008A3020008A30200082A
:10022000A3020008A3020008A3020008A30200081A
:10023000A3020008A3020008A3020008A30200080A
:10024000A3020008A3020008A3020008A3020008FA
:10025000A3020008A3020008A3020008A3020008EA
:10026000A3020008A3020008A3020008A3020008DA
:10027000A3020008A3020008A3020008A3020008CA
:10028000A3020008A3020008A3020008A3020008BA
:10029000A3020008A3020008A3020008A3020008AA
:1002A00002E000F000F8FEE772B6394880F30888F3
:1002B000384880F3098838484EF60851CEF20001DC
:1002C000086040F20000CCF200004EF63471CEF22D
:1002D00000010860BFF34F8FBFF36F8F40F2000043
:1002E000C0F2F0004EF68851CEF200010860BFF374
:1002F0004F8FBFF36F8F4FF00000E1EE100A4EF604
:100300003C71CEF200010860062080F31488BFF330
:100310006F8F02F057F903F071F94FF055301F4914
:100320001B4A91423CBF41F8040BFAE71C49194AA9
:1003300091423CBF41F8040BFAE71A491A4A1B4B99
:100340009A423EBF51F8040B42F8040BF8E7002034
:100350001749184A91423CBF41F8040BFAE702F0F2
:1003600075F903F0BFF9144C144DAC4203DA54F89C
:10037000041B8847F9E700F041F8114C114DAC42DD
:1003800003DA54F8041B8847F9E702F05DB900006E
:1003900000040024002400240000000800000024C1
:1003A000000400240840000800240024382400240D
:1003B0003824002450390024A0020008A0020008BC
:1003C000A0020008A00200082DE9F04F2DED108AD0
:1003D000C1F80CD0D0F80CD0BDEC108ABDE8F08F7D
:1003E000002383F311882846A047002001F066FD12
:1003F000FEE701F015FD00DFFEE7000038B51C4CFC
:100400006FF07403002523701C236570A570E570E0
:1004100025716571A571E57125726572A372E5722A
:1004200000F0BCFC20B10E2325726572A372E57248
:1004300002F06CF80F4B984217D00133984241F20A
:10044000883412BF002500240125002002F064F842
:100450000DB100F0B5F800F0E5FC00F023FC2046FB
:1004600000F06EF900F0ACF8F9E700242546ECE75F
:1004700038240024010007B008B500F0B5FBA0F156
:1004800020035842584108BD07B5054B02211B887F
:10049000ADF8043001A800F0F5FB03B05DF804FBF3
:1004A000E43C0008064991F8243033B100230822C7
:1004B000086A81F8243000F019BC0120704700BFA1
:1004C000582400242DE9F84F234C94F82430054695
:1004D000884617468BBB2E46DFF87C90002F38D01D
:1004E00094F824A0BAF1000F05D12022FF2148463C
:1004F000266200F085FCCAF10805BD4228BF3D46D2
:100500005FFA85FBAD0041462A4604EB8A0000F005
:100510004DFC94F82430A7EB0B079B445FFA8BFB50
:10052000BBF1080F2E44A844FFB284F824B0D5D103
:10053000FFF7B8FF0028D1D108E0266A06EB830652
:10054000B042C9D0FFF7AEFF0028C4D10020BDE8FB
:10055000F88F0120BDE8F88F5824002410B520231F
:1005600083F311881248C3680BB101F02DFD0023FD
:10057000104A0F484FF47A7101F0EAFC002383F32C
:1005800011880D4C236813B12368013B2360636815
:1005900013B16368013B6360084B1B7833B9636830
:1005A00023B9022000F000FC3223636010BD00BFBD
:1005B000442400245D0500088829002480240024A8
:1005C0002DE9F041544B554953F8042F013201D124
:1005D000BDE8F0818B42F7D1514C524B22689A42D0
:1005E00040F29880504B9B6803F1006303F50033A1
:1005F0009A4280F08F80002000F070FB4B4B02206D
:10060000187000F0CFFB4A4BD3F8E8200022C3F863
:10061000E820D3F81011C3F81021D3F81011D3F843
:10062000EC10C3F8EC20D3F81411C3F81421D3F85C
:100630001411D3F8F010C3F8F020D3F81811C3F850
:100640001821D3F81811D3F8801041F00061C3F8D5
:100650008010D3F8801021F00061C3F88010D3F827
:100660008010D3F8801041F00071C3F88010D3F8E7
:10067000801021F00071C3F88010D3F8803072B67A
:100680002C492D4B0B601D682468BFF34F8FBFF3BF
:100690006F8F2A4BC3F88420BFF34F8F5A6922F41F
:1006A00080325A61BFF34F8FD3F88020C2F3C9065E
:1006B000C2F34E325201B70743F6E07E02EA0E085B
:1006C00038463146013948EA000CB1F1FF3FC3F822
:1006D00074C200F14040F5D1203A12F1200FEDD163
:1006E000BFF34F8FBFF36F8FBFF34F8FBFF36F8F8A
:1006F0005A6922F400325A610022C3F85022BFF333
:100700004F8FBFF36F8F202383F31188AD4685F39E
:1007100008882047BDE8F081FCFF01081C000208A2
:1007200004000208FFFF010838240024802400246C
:100730000044025808ED00E00000020800ED00E06F
:100740002DE9F04FB54C97B020228246FF210EA82C
:10075000A56800F055FBB24A1378A046A3B9B1488A
:100760000121C3601170202383F31188C3680BB18A
:1007700001F02AFC0023AC4AAA484FF47A7101F038
:10078000E7FB002383F31188DFF8BCB2BAF1000F56
:1007900001D0CBF800A0A54F00243C70CBF804405A
:1007A0002646012000F0FEFABAF1000F00F0E081C9
:1007B000DBF80030002B40F0DB8117B0BDE8F08F94
:1007C0000220FFF759FE002840F0D081984B1B888B
:1007D000ADF82430022109A800F054FAE1E74FF403
:1007E0007A7000F001FA031E0193EFDB0220FFF79D
:1007F00043FE81460028E9D0019B581E0428E5D815
:10080000DFE800F0030C0F12150016A8052340F8CE
:10081000343D042100F036FA4C4650E004217F4874
:10082000F8E704218348F5E704218348F2E71C2414
:10083000204600F055FA04340990042109A800F07C
:1008400021FA2C2CF4D1E7E7002EBFD0002CBDD02C
:100850000220FFF711FE064610B901242646B5E72F
:10086000012000F03BFA0220387000F09BFA0024CF
:10087000E3B21846019300F041FA814648B1019B6A
:10088000184600F04BFA01340028F1D134466B4B86
:100890009DE7012302203B7000F082FA4D46D8F814
:1008A00008309D4206D2284600F01AFA0130EDD1F8
:1008B0000435F4E700253D70CBF80450344600F0D1
:1008C000A7FAFFF7E1FD4EE1002E3FF47FAF002CC9
:1008D0003FF47CAF0220387000F064FA322000F060
:1008E00083F9041EB9DB14F00306B6D1D8F808204A
:1008F0002B199342B1D8B4F5807FAED8DFF8409180
:10090000A6420CDA4FF47A7000F06EF90390039B64
:10091000002BA2DB039B06F809300136F0E7C82064
:10092000FFF7AAFD0646002897D01F2D11D8C5F164
:100930002009A14528BFA1460EAB25F003004A4679
:100940003F49184400F032FA4A46FF213C4800F083
:1009500057FA4FEAA4095FFA89F239492846FFF7A6
:10096000B1FD0446002891D005EB89050646A6E7AF
:100970000220FFF781FD00283FF428AFFFF792FD2A
:1009800000283FF423AF4FF0000AD146D8F80830D2
:100990009A453CD2BAF11F0F1CD80E9B013319D0D7
:1009A0002AF0030316AA134453F8203C099325495F
:1009B0004B68A3B1002209A8135C83EA0903DBB2E8
:1009C000013251F82330042A83EA1929F4D10AF1BB
:1009D000040ADBE7504600F083F90990E7E71A467E
:1009E000082012F0010F4FEA52021FBF82F06D4241
:1009F00082F4380282F4034282F020020138F0D1FE
:100A000041F823200133B3F5807FE8D1D2E716A85F
:100A1000042140F8489D00F035F950E738240024BF
:100A200084250024442400245D050008802400243B
:100A3000E63C00083C24002440240024E83C000854
:100A400084240024882500248829002416A8002353
:100A500040F8343D642100F0F1F800287FF4B6AE90
:100A60000220FFF709FD00283FF4B0AE099800F01E
:100A700067F916AB43F8440D04211846CBE716A8D6
:100A8000002340F8343D642100F0D8F800287FF4BA
:100A90009DAE0220FFF7F0FC00283FF497AE0998C6
:100AA00000F050F916AB43F8400DE5E70220FFF7E0
:100AB000E3FC00283FF48AAE00F04AF916AB43F895
:100AC0003C0DD9E70220FFF7D7FC00283FF47EAEAB
:100AD00009A9142000F042F9814616A8042140F823
:100AE000389D00F0CFF8494609A894E74FF47A7092
:100AF000FFF7C2FC00283FF469AEFFF7D3FC0028E3
:100B00003FF4C5AE0E9B01330CD008220EA9002085
:100B1000FFF7D8FC00283FF4BAAE2022FF210EA830
:100B200000F06EF9FFF7B0FC2E4801F0CDF944E675
:100B300016A8002340F8343D642100F07FF8002817
:100B40007FF444AE0220FFF797FC00283FF43EAE4E
:100B5000FFF79AFC41F2883001F0B6F9099800F0ED
:100B600093F900F055F94FF0000A1AE60646A6E69A
:100B7000002000F039F80390039B002BFFF614AE21
:100B8000012000F00DF9039B213B122B3FF609AE2B
:100B900001A252F823F000BFC1070008DF070008D8
:100BA00049080008A3070008A3070008A3070008D6
:100BB000C9080008A3070008710900084D0A0008C9
:100BC0007F0A0008AD0A0008A3070008C50A00084C
:100BD000A3070008ED0A0008BF080008A3070008E3
:100BE000310B0008A086010037B5114B1A7801328D
:100BF000D2B20024012A01468DF8074011D80D48D1
:100C000003681D6A4FF47A734B4301220DF107010B
:100C1000A847012805D1084B9DF807001C7003B0B8
:100C200030BD4FF4FA7001F04FF94FF0FF30F6E7A6
:100C3000002400245C2E0024AC29002438B50E4B7F
:100C40001A780132D2B2012A05460ED80B48036841
:100C50001C6A4FF47A734B4304222946A0470428A8
:100C600003D1074B0020187038BD4FF4FA7001F023
:100C70002BF94FF0FF3038BD002400245C2E0024F7
:100C8000AC29002430B4054C2368DD69044B0A46C6
:100C9000AC460146204630BC604700BF5C2E0024B5
:100CA000A0860100F8B501F055FB094C094E0A4F2A
:100CB0002070002530682378834207D901F046FB75
:100CC000336805440133BD423360F3D9F8BD00BF3A
:100CD000AD29002490290024FFFF010001F002BC8F
:100CE00000F1006000F500300068704700F100601E
:100CF000920000F5003001F097BB0000054B1A6828
:100D0000054B1B789B1A834202D9104401F01EBB8D
:100D10000020704790290024AD29002438B5074DE4
:100D200004462868204401F017FB28B928682044AD
:100D3000BDE8384001F022BB38BD00BF9029002437
:100D400000207047014BC058704700BF00E8F11FFA
:100D5000014B1868704700BF0010005C70B50E4B67
:100D60005C6893F9086001380A18013C0B4693420D
:100D70000FD214F9015F581C1DB1034600F8015C45
:100D8000F5E72C2482421C7001D9981C5E70401A31
:100D900070BD1846FBE700BF042400240020704704
:100DA00070470000704700007047000010B5002336
:100DB000934203D0CC5CC4540133F9E710BD00006A
:100DC00030B5441E14F9010F0B4660B193F9005081
:100DD000854201F1010106D11AB993F90020801A68
:100DE00030BD013AEEE7002AF7D1104630BD0000D1
:100DF00002460346981A13F9011B0029FAD17047DD
:100E000002440346934202D003F8011BFAE77047FD
:100E1000024B1A78024B1A70704700BFAC290024AD
:100E20000024002438B5134D134C284600F07EFBF7
:100E30002146284600F0A6FB23681048D3F89020EE
:100E4000D2F8043843F00203C2F8043801F03CF849
:100E50000B49206800F0A6FC2368D3F89020D2F854
:100E6000043823F00203C2F80438064B4FF4E13291
:100E70001A6038BD5C2E0024A03D000840420F00DF
:100E8000F03D00089429002470470000FEE70000B0
:100E900000B59BB0EFF3098168226846FFF786FF33
:100EA000EFF30583034B9A6B9A6A9A6A9A6A9A6A75
:100EB0009B6AFEE700ED00E000B59BB0EFF309810F
:100EC00068226846FFF772FFEFF30583034B9A6AC7
:100ED0009A6A9A6A9A6A9A6A9B6AFEE700ED00E04B
:100EE00000B59BB0EFF3098168226846FFF75EFF0B
:100EF000EFF30583034B5A6B9A6A9A6A9A6A9A6A65
:100F00009B6AFEE700ED00E0024A136843F0C0036D
:100F10001360704700780040044B5A6810439A6889
:100F200058600AB1181D1047704700BFB02900244F
:100F30002DE9F84F404EF56D2F68EC692C622107C2
:100F400018D014F0080F0CBF00208020E20748BF23
:100F500040F02000A30748BF40F04000610748BFB1
:100F600040F48070202383F31188FFF7D5FF00231E
:100F700083F31188E20509D5202383F311884FF408
:100F80000070FFF7C9FF002383F31188DFF8A8A0E2
:100F90004FF020094FF0000B14F0200832D13B062F
:100FA00015D5DFF898A04FF0200920060FD589F35A
:100FB0001188504600F09AF9002830DA0820FFF72F
:100FC000ABFF27F080032B60002383F311887906A1
:100FD0000DD562060BD5202383F31188F26C336D97
:100FE0009A4201D1336C03BB002383F31188E306DB
:100FF00004D5B26E13690BB150699847BDE8F84F3C
:1010000001F0B2BA89F31188AB8C96F8641050469F
:10101000194000F0F7F98BF31188EC69BCE780B256
:10102000288588F31188EC69BFE7102027F0400776
:10103000FFF772FF2F60D7E7B0290024E8290024CA
:1010400013B5104C204600F0D1F904F114000094BF
:1010500000234FF400720C4900F092F804F13800BC
:1010600000940A4B0A494FF4007200F00BF9094B47
:10107000E365094B23660C21522002B0BDE8104005
:1010800000F00CB8B02900241C2A0024090F000825
:101090001C2C00240078004000366E0100F16043F3
:1010A00000F01F02400903F5614309018000C9B245
:1010B00000F1604083F8001300F561400123934084
:1010C000C0F8803103607047F8B51546826806693C
:1010D000AA420B46816938BF8568761AB542044634
:1010E00007D218462A46FFF761FEA3692B44A36185
:1010F0000DE011D932461846FFF758FEAF1B3A46AD
:10110000E1683044FFF752FEE2683A44A261A36806
:101110005B1BA3602846F8BD18462A46FFF746FE2B
:10112000E368E4E783682DE9F041044693421546FD
:10113000266938BF85684069361AB5420F4606D21F
:101140002A46FFF733FE63692B4463610DE012D931
:101150003246A5EB0608FFF729FE4246B919E068BA
:10116000FFF724FEE26842446261A3685B1BA36050
:101170002846BDE8F0812A46FFF718FEE368E4E759
:1011800010B50A440024C361029B00604060846083
:10119000C160816141610261036210BD08B582696D
:1011A0004369934201D1826882B9826801328260C8
:1011B0005A1C42611970426903699A4201D3C3689B
:1011C0004361002100F09CFE002008BD4FF0FF307D
:1011D00008BD000070B5202304460E4683F3118835
:1011E000A568A5B1A368A269013BA360531CA361D4
:1011F00015782269934224BFE368A361E3690BB1C8
:1012000020469847002383F31188284670BD314655
:10121000204600F065FE0028E2DA85F3118870BDF3
:101220002DE9F74F05460F4690469A46D0F81C9098
:10123000202686F311884FF0000B144664B1224635
:1012400039462846FFF740FF034668B9514628460D
:1012500000F046FE0028F1D0002383F31188A8EBAC
:10126000040003B0BDE8F08FB9F1000F03D0019086
:101270002846C847019B8BF31188E41A1F4486F364
:101280001188DBE7C16081614161C3611144009B4A
:10129000006040608260016103627047F8B50446F7
:1012A0000E461746202383F31188A568A5B1A368CD
:1012B000013BA36063695A1C62611E702369626905
:1012C0009A4224BFE3686361E3690BB12046984703
:1012D000002080F31188F8BD3946204600F000FE5A
:1012E0000028E2DA85F31188F8BD000083694269BD
:1012F0009A4210B501D182687AB98268013282605F
:101300005A1C82611C7803699A4201D3C3688361C5
:10131000002100F0F5FD204610BD4FF0FF3010BD5C
:101320002DE9F74F05460F4690469A46D0F81C9097
:10133000202686F311884FF0000B144664B1224634
:1013400039462846FFF7EEFE034668B9514628465F
:1013500000F0C6FD0028F1D0002383F31188A8EB2C
:10136000040003B0BDE8F08FB9F1000F03D0019085
:101370002846C847019B8BF31188E41A1F4486F363
:101380001188DBE7026843681143016003B1184725
:10139000704700001430FFF743BF00004FF0FF33E9
:1013A0001430FFF73DBF00003830FFF7B9BF000031
:1013B0004FF0FF333830FFF7B3BF00001430FFF7B2
:1013C00009BF00004FF0FF311430FFF703BF0000EA
:1013D0003830FFF763BF00004FF0FF323830FFF7BF
:1013E0005DBF000000207047FFF72ABE044B03607A
:1013F000002343608360C36001230374704700BF10
:10140000FC3C000838B5C36904460D461BB90421ED
:101410000844FFF7B7FF294604F11400FFF7BEFEAA
:10142000002806DA201D4FF48061BDE83840FFF740
:10143000A9BF38BD026843681143016003B1184772
:101440007047000013B5446BD4F894341A681178CF
:10145000042915D1217C022912D11979128901237D
:101460008B4013420CD101A904F14C0001F03AFF6A
:10147000D4F89444019B21790246206800F0EAF9EF
:1014800002B010BD143001F0BDBE00004FF0FF33BC
:10149000143001F0B7BE00004C3001F08FBF0000E7
:1014A0004FF0FF334C3001F089BF0000143001F0E1
:1014B0008BBE00004FF0FF31143001F085BE0000FC
:1014C0004C3001F05BBF00004FF0FF324C3001F0B8
:1014D00055BF0000D0F8942438B513681978042952
:1014E000054601D0012038BD017C0229FAD11279CC
:1014F0005C89012090400440F4D105F1140001F012
:101500001DFE02460028EDD0D5F894544FF48073A8
:101510002868697900F08CF9204638BD406BFFF7E8
:10152000D9BF000000207047704700007FB5124B04
:101530000360002343608360C360012502260F4BD4
:10154000057404460290019300F184022946009636
:101550004FF48073143001F0CDFD094B01930294D8
:1015600000964FF4807304F52372294604F14C0071
:1015700001F094FE04B070BD243D00081D15000864
:10158000451400080A68202383F311880B790B3374
:1015900042F823004B79133342F823008B7913B1BF
:1015A0000B3342F8230002230374C0F89414002381
:1015B00083F311887047000038B5037F044613B1E8
:1015C00090F85430ABB9201D01250221FFF732FFFE
:1015D00004F1140025776FF0010100F09DFC84F800
:1015E000545004F14C006FF00101BDE8384000F0A8
:1015F00093BC38BD10B5012104460430FFF71AFF33
:101600000023237784F8543010BD000038B5044619
:101610000025143001F086FD04F14C00257701F01F
:1016200055FE201D84F854500121FFF703FF20468A
:10163000BDE83840FFF74EBF90F8803003F06003FC
:10164000202B19D190F88120212A0AD0222A4FF08C
:1016500000030ED0202A0FD1084A42670722826772
:1016600004E0064B4367072383670023C367012019
:10167000704743678367F9E7002070471024002410
:10168000D0F8943437B51A681178042904461AD171
:10169000017C022917D11979128901238B40134249
:1016A00011D100F14C05284601F0D0FE58B101A936
:1016B000284601F017FED4F89444019B2179024694
:1016C000206800F0C7F803B030BD000001F10B0343
:1016D000F7B550F8234005460E46F4B1202383F3B6
:1016E000118805EB8607201D0821FFF7A3FEFB6884
:1016F0005B691B684C3413B1204601F001FE01A95F
:10170000204601F0EFFD024648B1019B31462846D4
:1017100000F0A0F8002383F3118803B0F0BDFB684C
:101720005A691268002AF5D01B8A013B1340F1D197
:1017300005F18002EAE70000133138B550F8214086
:10174000DCB1202383F31188D4F8942413685279F0
:1017500003EB8203DB689B695D6845B10421601877
:10176000FFF768FE294604F1140001F0F1FC204661
:10177000FFF7B0FE002383F3118838BD70470000E7
:1017800000F0ECBF012303700023436000F130023E
:1017900000F1500142F8043B8A42D361FAD103813F
:1017A0004381704738B50446202383F31188002510
:1017B000416000F10C0300F1300243F8045B9342F6
:1017C000FBD1204600F0ECFF0223237085F3118843
:1017D00038BD000070B500EB810305465069DA6042
:1017E0000E46144618B110220021FFF709FBA0692C
:1017F00018B110220021FFF703FB31462846BDE84F
:10180000704001F0DFB80000038903F00103038199
:10181000438903F00103438100F1300200F110031A
:10182000002143F8041B9342FBD101F063B900008F
:10183000F0B400EB81044789E4680125A4698D4078
:101840003D43458123600023A2606360F0BC01F04A
:101850007FB90000F0B400EB81040789E46801253A
:1018600064698D403D43058123600023A26063606D
:10187000F0BC01F0F7B90000022310B5037000239B
:101880000446A0F8883080F88A3080F88B300381D5
:10189000438100F10C0200F1300142F8043B8A421E
:1018A000FBD184F87030204601F020F863681B6893
:1018B00023B120460021BDE81040184710BD0000AC
:1018C000436802781B6880F88C20052202700BB1F7
:1018D0000421184770470000436890F88C201B686B
:1018E00002700BB1052118477047000090F8703066
:1018F00070B5044613B1002380F8703004F1800203
:10190000204601F01BF963689B6863BB94F8805024
:1019100015F0600615D194F8813005F07F0545EA91
:10192000032540F202339D4200F00E815BD8022D68
:1019300000F0DC803FD8002D00F08780012D00F002
:10194000CF800021204601F0B1FB0021204601F0AC
:10195000A1FB63681B6813B1062120469847062344
:1019600084F8703070BD204698470028CED094F897
:10197000872094F8863043EA0223A26F934238BF4F
:10198000A36794F98030A56F002B4FF0200380F2FD
:10199000FD80002D00F0EC80092284F8702083F394
:1019A00011880021A36F626F2046FFF753FF0023C9
:1019B00083F3118870BDB5F5817F00F0B180B5F576
:1019C000407F49D0B5F5807FBBD194F88230012BA0
:1019D000B7D1B4F8883023F00203A4F888306667E2
:1019E000A667E667C3E740F201639D421ED8B5F5DE
:1019F000C06F3BD2B5F5A06FA3D1B4F88030B3F57A
:101A0000A06F0ED194F8823084F88A30204600F01E
:101A1000CBFF63681B6813B101212046984703235D
:101A2000237000236367A367E367A0E7B5F5106F32
:101A300032D040F602439D4252D0B5F5006F80D1BE
:101A400004F18B036367012324E004F188036367D7
:101A50000223A367E5678AE794F88230012B7FF4BD
:101A600070AFB4F8883043F00203B6E794F88520ED
:101A7000616894F884304D6894F8831043EA022337
:101A8000204694F88220A84700283FF45AAF4368C4
:101A900063670368A367A4E72378042B10D120238E
:101AA00083F311882046FFF7AFFE86F31188636841
:101AB00084F88B601B68032121700BB12046984786
:101AC00094F88230002BACD084F88B300423237040
:101AD00063681B68002BA4D0022120469847A0E72A
:101AE000374B63670223A36700239DE794F88410B4
:101AF00011F0800F204601F00F010ED001F010F818
:101B0000012806D002287FF41CAF2E4B6367A06724
:101B100067E72D4B6367A56763E700F0F3FFEFE727
:101B200094F88230002B7FF40CAF94F8843013F0DB
:101B30000F013FF476AF1A06204602D501F0CEFA27
:101B40006FE701F0BFFA6CE794F88230002B7FF466
:101B5000F8AE94F8843013F00F013FF462AF1B0627
:101B6000204602D501F0A2FA5BE701F093FA58E7AC
:101B7000142284F8702083F311882B462A462946C4
:101B80002046FFF755FE85F3118870BD5DB1152223
:101B900084F8702083F311880021A36F626F2046C0
:101BA000FFF746FE03E70B2284F8702083F31188C9
:101BB0002B462A4629462046FFF74CFEE3E700BFA6
:101BC000543D00084C3D0008503D000838B590F8E1
:101BD00070300446152B29D8DFE803F03E2828286A
:101BE00028283E28280B293928282828282828286A
:101BF0003E3E90F8871090F88620836F42EA0122DB
:101C00009A4214D9C268128AB3FBF2F502FB153569
:101C10006DB9202383F311882B462A462946FFF706
:101C200019FE85F311880A2384F8703038BD142317
:101C300084F87030202383F3118800231A46194654
:101C40002046FFF7F5FD002383F3118838BDC36FED
:101C500003B198470023E7E7002101F027FA0021AC
:101C6000204601F017FA63681B6813B1062120466D
:101C700098470623D8E7000090F87020152A38B559
:101C8000044622D80123934040F6416213421DD1FD
:101C900013F480150FD19B0217D50B2380F87030F9
:101CA000202383F311882B462A462946FFF7D2FDCD
:101CB00085F3118838BDC3689B695B682BB9C36F16
:101CC00003B19847002384F8703038BD002101F03B
:101CD000EDF90021204601F0DDF963681B6813B1BE
:101CE0000621204698470623EDE70000024B00221C
:101CF0001B605B609A6070471C2E002400230374F5
:101D00008268054B1B6899689142FBD25A68036050
:101D100042601060586070471C2E002408B52023D4
:101D200083F31188037C032B05D0042B0DD02BB932
:101D300083F3118808BD436900221A604FF0FF3316
:101D40004361FFF7DBFF0023F2E790E80C001A6025
:101D500002685360F2E70000002303748268054BB9
:101D60001B6899689142FBD85A6803604260106012
:101D7000586070471C2E0024054B196908741868B8
:101D800002681A605360186101230374FEF71CBBDC
:101D90001C2E002430B54B1C87B005460A4C10D0D1
:101DA00023690A4A01A800F0D3F82846FFF7E4FFA8
:101DB000049B13B101A800F007F92369586907B023
:101DC00030BDFFF7D9FFF8E71C2E00241D1D0008C9
:101DD00038B50C4D41612B6981689A68914204467F
:101DE00003D8BDE83840FFF789BF1846FFF786FFE4
:101DF00001232C61014623742046BDE83840FEF7DC
:101E0000E3BA00BF1C2E0024044B1A681B699068BB
:101E10009B68984294BF0020012070471C2E00242C
:101E200010B5084C236820691A68226054600122AA
:101E300023611A74FFF790FF01462069BDE8104046
:101E4000FEF7C2BA1C2E0024826002220274002215
:101E5000427470478368A3F17C0243F80C2C02693A
:101E600043F83C2C426943F8382C074A43F81C2CB1
:101E7000C26843F8102C022203F8082C002203F851
:101E8000072CA3F118007047E103000810B52023C8
:101E900083F31188FFF7DEFF00210446FFF798FF68
:101EA000002383F31188204610BD0000024B1B69FC
:101EB00058610F20FFF760BF1C2E0024202383F3FE
:101EC0001188FFF7F3BF000008B50146202383F314
:101ED00011880820FFF75EFF002383F3118808BDF7
:101EE00049B1064B42681B6918605A601360436031
:101EF0000420FFF74FBF4FF0FF3070471C2E002427
:101F00000368984206D01A6802605060596118460A
:101F1000FFF7F4BE7047000038B504460D46206850
:101F2000844200D138BD036823605C604561FFF7DF
:101F3000E5FEF4E7054B03F114025A619A614FF094
:101F4000FF32DA6100221A62704700BF1C2E0024A3
:101F5000F8B503614FF08043C2605C6A194B1A46C2
:101F6000022952F8145F38BF0221954206461F46E7
:101F70000AD1586198611C6205604560816008194A
:101F8000BDE8F84001F084BA186AAB68241A0C194D
:101F900002D3E41A2D6804E09C4202D2204401F0EE
:101FA00085FAAB689C42F4D86B68736035601E603C
:101FB0006E60B460A9684FF0FF33091BA960FB6134
:101FC000F8BD00BF1C2E002410B41B4C234653F850
:101FD000141F814210D0416802680A600268516093
:101FE0009A424FF00001C16003D0936881680B44AE
:101FF00093605DF8044B70470A68626100209A4262
:102000005360C86003D15DF8044B01F049BA93688E
:102010008868034493604FF08042206A526A121A23
:102020009342E6D9991A012998BF931C18445DF888
:10203000044B01F03BBA00BF1C2E00240020704767
:10204000FEE70000704700004FF0FF3070470000CF
:10205000022906D0032906D00129064818BF00200E
:10206000704705487047032A9ABF044800EBC20036
:10207000002070474C3E0008003E00081824002451
:1020800070B5044608460D46FEF7B2FEC6B22046BD
:10209000013403780BB9184670BD32462946FEF765
:1020A0008FFE0028F3D1012070BD00002DE9F04F14
:1020B00081469BB008460C461646FEF799FE3C4901
:1020C000C5B22046FFF7DCFF08B10335EDB2394950
:1020D0002046FFF7D5FF08B11035EDB2632D01AFF3
:1020E0000CD8DFF8DCA0DFF8DCB03D4694F80080C7
:1020F000B8F1000F1CD185F8008003E02146384676
:1021000001F0E8FD3846FEF773FEC0B2431C5B00E9
:1021100089E84800337003237370002302361946A0
:10212000DAB2904206F102063AD81BB0BDE8F08F51
:10213000B8F1250F2FD107221D492046FEF740FE9A
:1021400058B9DBF800202A60DBF804206A60BBF88D
:1021500008202A8107340A35C8E708221549204695
:10216000FEF72EFEB8B91448AA1C10F8011F134B35
:102170004FEA111E01F00F011EF80AE011F80A10D3
:1021800002F802EC984202F8011C02F10202ECD1C2
:1021900018350834AAE785F8008001340135A5E731
:1021A000FA5C06F8022C06F8011C0133B8E700BF00
:1021B000A83D0008B03D0008FFE7F11F0BE8F11F44
:1021C000C43D0008B93D000808B5202383F31188F9
:1021D0000348FFF755FA002383F3118808BD00BFB9
:1021E0005C2E002410B50446052916D8DFE801F05E
:1021F00016150316161D202383F311880E4A01219C
:10220000FFF7E8FA20460D4A0221FFF7E3FA0C48EF
:10221000FFF7FCF9002383F3118810BD202383F31B
:1022200011880748FFF7C8F9F4E7202383F31188E2
:102230000348FFF7DFF9EDE7583D00087C3D000853
:102240005C2E002438B50C4D0C4C0D492A4604F187
:102250000800FFF72BFF05F1CA0204F1100009493D
:10226000FFF724FF05F5CA7204F118000649BDE81E
:102270003840FFF71BBF00BF24330024182400247C
:10228000D83D0008E23D0008B03D0008BFF34F8F85
:10229000044B1A695107FCD1D3F810215207F8D129
:1022A000704700BF0020005208B50D4B1B78ABB93A
:1022B000FFF7ECFF0B4BDA68D10741BF0A4A5A60BF
:1022C00002F188325A60D3F80C21D20741BF064A86
:1022D000C3F8042102F18832C3F8042108BD00BF0D
:1022E00082350024002000522301674508B5114BB8
:1022F0001B78F3B9104B1A69510742BFDA6842F0F4
:102300004002DA60D3F81021520742BFD3F80C2103
:1023100042F04002C3F80C21FFF7B8FF064BDA6821
:1023200042F00102DA60D3F80C2142F00102C3F856
:102330000C2108BD82350024002000520E289ABFCF
:1023400000F5806040040020704700004FF400302A
:10235000704700000F2070470E2808B50BD8FFF714
:10236000EDFF00F500330268013204D104308342EE
:10237000F9D1012008BD002008BD00000E2810B5CD
:1023800004464AD8FFF782FFFFF78EFF24484FF03C
:10239000FF33072C4361C0F8143124D80361FFF7E1
:1023A00075FF230243F02403C360C36843F0800336
:1023B000C36003695A07FCD4FFF768FF2046FFF7A4
:1023C000BDFF00F50033BFF34F8F164A984220D36C
:1023D000BFF34F8FBFF36F8FFFF788FF2046BDE835
:1023E0001040FFF7B9BFC0F81031FFF74FFFA4F15D
:1023F00008031B0243F02403C0F80C31D0F80C3161
:1024000043F08003C0F80C31D0F810315B07FBD4E7
:10241000D2E7C2F85C022030D8E7002010BD00BF30
:102420000020005200ED00E02DE9F84F42EA0003E1
:10243000DB0605460E46174643D1FFF735FFDFF8AA
:102440009880DFF89890DFF898A034463B1B33441F
:102450001F2B04D8FFF74AFF0120BDE8F88F1C4A64
:102460001C4805F1784393429ABF5046C346CB4679
:10247000FFF70CFF4FF0FF33CBF80030036843F059
:102480000203036004F11C01231F53F804EFEA1850
:10249000121B8B42C2F800E0F7D1BFF34F8FFFF75A
:1024A000F5FE4FF0FF33CBF80030036823F0020352
:1024B000036020222146284601F0FCFB20B1FFF7F3
:1024C00015FF0020BDE8F88F20352034BEE700BF9F
:1024D000FFFF0F000C210052142000521421005263
:1024E0000C20005210B5084C237828B153B9FFF7DF
:1024F000DBFE0123237010BD23B12070BDE8104026
:10250000FFF7F4BE10BD00BF82350024014B186DEB
:10251000704700BF00400058084B1A6F120405D4E2
:102520001A6F1A671A6F42F400421A67044A136856
:1025300043F480731360034B1865704700440258DE
:102540000048025800400058064A536823F001032F
:102550005360EFF30983683383F30988002383F31F
:102560001188704730EF00E010B5202383F3118805
:10257000104B5B6813F4006318D0F1EE103AEFF3E0
:1025800009844FF0807344F84C3C0B4BDB6844F8F3
:10259000083CA4F1680383F30988FFF735FC18B100
:1025A000064B44F8503C10BD054BFAE783F3118805
:1025B00010BD00BF00ED00E030EF00E0F3030008C5
:1025C000F6030008F0B5BFF34F8FBFF36F8F1D4BBD
:1025D0000021C3F85012BFF34F8FBFF36F8F5A69BA
:1025E00042F400325A61BFF34F8FBFF36F8FC3F8CD
:1025F0008410BFF34F8FD3F88020C2F3C904C2F315
:102600004E325201A50743F6E07602EA060E28464E
:1026100021464EEA00070139C3F860724F1C00F1F1
:102620004040F6D1203A12F1200FEED1BFF34F8F88
:102630005A6942F480325A61BFF34F8FBFF36F8FF4
:10264000F0BD00BF00ED00E0FEE70000084A094BC6
:1026500009498B4204D3094A0021934205D37047AC
:1026600052F8040F43F8040BF3E743F8041BF4E7B4
:102670003C400008503900245039002450390024CF
:10268000D0F8943030B500229D68D0F890401146C3
:102690004FF0FF3004EB421301329542C3F80019AA
:1026A000C3F81019C3F80809C3F8001BC3F8101BBE
:1026B000C3F8080BEED24FF00113C4F81C3830BD3C
:1026C00000EB81032DE9F04FD3F80CE0DEF8144065
:1026D0004F1CD4F800C03F034FEA41186568D0F89A
:1026E000902065450AD3D2F83438012000FA01F170
:1026F00023EA0101C2F83418BDE8F08FBEF810607B
:10270000ACEB0503B34228BF334602EB0806D6F80C
:102710001869B6B2B3EB860F13D8A6683A44A6F18F
:10272000040A99465AF804BFC2F800B0B9F1040F80
:1027300002D9A9F10409F5E71E442B44A6606360A1
:10274000CCE70020BDE8F08F890141F02001016154
:1027500003699B06FCD4122000F036BF10B50A4C6A
:102760002046FFF70FF8094BC4F89030084BC4F827
:102770009430084C2046FFF705F8074BC4F890301A
:10278000064BC4F8943010BD843500240000084086
:10279000903E000820360024000004409C3E0008C3
:1027A0000378012B70B505465DD1494BD0F89040B8
:1027B000984259D1474BD3F8D82042F00062C3F871
:1027C000D820D3F8002142F00062C3F80021D3F8EA
:1027D0000021D3F8802042F00062C3F88020D3F8B3
:1027E000802022F00062C3F88020D3F880300E21D0
:1027F0006520FEF753FC384BE360384BC4F80038D3
:102800000023C4F8003EC0232360D5F890604FF445
:102810000413A3633369002BFCDA012333610C201A
:1028200000F0D2FE3369DB07FCD4122000F0CCFEAE
:102830003369002BFCDA0026A6602846FFF720FF4C
:102840006B68C4F81068DB68C4F81468C4F81C68C6
:10285000002B3AD1224BA3614FF0FF336361A36891
:1028600043F00103A36070BD1E4B9842C8D1194BC1
:10287000D3F8D82042F00072C3F8D820D3F8002152
:1028800042F00072C3F80021D3F80021D3F8802071
:1028900042F00072C3F88020D3F8802022F000724A
:1028A000C3F88020D3F88020D3F8D82022F08062AB
:1028B000C3F8D820D3F8002122F08062C3F80021A9
:1028C000D3F800310E214D2093E7074BC3E700BF3B
:1028D00084350024004402584014004003002002C4
:1028E000003C30C020360024083C30C0F8B5D0F899
:1028F0009040054600212046FFF726FFD5F89410AA
:1029000000234FF001128F68C4F834384FF000668E
:10291000C4F81C284FF0FF3004EB431201339F42F0
:10292000C2F80069C2F8006BC2F80809C2F8080BC7
:10293000F2D20B68D5F89020C5F898306362102366
:102940001361166916F01006FBD1122000F03CFE50
:10295000D4F8003823F4FE63C4F80038A36943F4C4
:10296000402343F01003A3610923C4F81038C4F8CE
:1029700014380B4BEB604FF0C043C4F8103B094BCD
:10298000C4F8003BC4F81069C4F80039D5F8983091
:1029900003F1100243F48013C5F89820A362F8BD38
:1029A0006C3E000840800010D0F8902090F88A100B
:1029B000D2F8003823F4FE6343EA0113C2F800386A
:1029C000704700002DE9F0410EB200EB86080D467D
:1029D000D8F80C100F6807F00303022B53D0032B19
:1029E00053D03F4A3F4F012B18BF1746D0F89040B5
:1029F0004FEA451E04EB0E030022C3F8102B8A6930
:102A000005F1100C002A42D04A8A05F158035B01F7
:102A10003A43E2500123D4F81C2803FA0CF3134381
:102A2000A6444A69C4F81C380023CEF8103905F1D1
:102A30003F03002A3BD00A8A898B9208012988BF6C
:102A40004A43D0F8981004EB8303561841EA024237
:102A5000C0F8986029465A602046FFF775FED8F8FE
:102A60000C301B8A43EA85531F4305F148035B0181
:102A7000E7500123D4F81C2803FA05F51543C4F8E0
:102A80001C58BDE8F081184FB0E7184FAEE704EBD3
:102A90004613D3F8002B22F40042C3F8002BD4F8DD
:102AA0001C28012303FA0CF322EA0303B8E704EB22
:102AB00083030F4A5A6004EB461629462046FFF767
:102AC00043FED6F8003923F40043C6F80039D4F8A1
:102AD0001C38012202FA05F523EA0505CFE700BFFD
:102AE00000800010008004100080081000800C108E
:102AF00000040002D0F894201268C0F89820FFF774
:102B0000BFBD00005831D0F8903049015B5813F434
:102B1000004004D013F4001F14BF012002207047AE
:102B20004831D0F8903049015B5813F4004004D08C
:102B300013F4001F14BF01200220704700EB810135
:102B4000CB68196A0B6813604B68536070470000CC
:102B500000EB810330B5DD68AA691368D36019B949
:102B6000402B84BF402313606B8A1468D0F89020F8
:102B70001C44013CB4FBF3F46343033323F003032D
:102B800002EB411043EAC44343F0C043C0F8103B9A
:102B90002B6803F00303012B09B20ED1D2F80838D9
:102BA00002EB411013F4807FD0F8003B14BF43F0D8
:102BB000805343F00053C0F8003B02EB4112D2F8BF
:102BC000003B43F00443C2F8003B30BD2DE9F04127
:102BD000D0F8906006EB41130546D3F8087BC3F8A4
:102BE000087B3A070C4608D5D6F814381B0704D5DD
:102BF00000EB8103DB685B689847FA072FD5D6F8AE
:102C00001438DB072BD505EB8403D968CCB98B6965
:102C1000488A5E68B6FBF0F200FB12628AB9186857
:102C2000DA6890420DD2121A83E81400202383F34D
:102C3000118821462846FFF78BFF84F31188BDE8F1
:102C4000F081012303FA04F26B8923EA02036B810A
:102C5000CB6823B121462846BDE8F0411847BDE8BE
:102C6000F081000000EB810370B5DD68D0F8903092
:102C70006C692668E6604A0156BB1A444FF400208E
:102C8000C2F810092A6802F00302012A0AB20ED122
:102C9000D3F8080803EB421410F4807FD4F800093D
:102CA00014BF40F0805040F00050C4F8000903EB1E
:102CB0004212D2F8000940F00440C2F80009D3F8EB
:102CC0003408012202FA01F10143C3F8341870BD3F
:102CD00019B9402E84BF4020206020682E8A8419B4
:102CE00040F00050013C1A44B4FBF6F440EAC44002
:102CF000C6E700002DE9F041D0F8906006EB4113E3
:102D00000446D3F80879C3F80879FB070D461CD5AB
:102D1000D6F81038DA0718D500EB8103D3F80CE0A9
:102D2000DEF81430D3F800C0DA6894451BD2A2EB69
:102D30000C024FF000081A60C3F80480202383F3CC
:102D40001188FFF78FFF88F311883B0618D5D6F856
:102D500034280123AB40134212D029462046BDE857
:102D6000F041FFF7ADBC012303FA01F2038923EA26
:102D700002030381DEF80830002BE6D09847E4E731
:102D8000BDE8F0812DE9F047D0F890506E69AB694D
:102D90001E40F10404466E6103D5BDE8F047FEF71E
:102DA0006BBD002E11DAD5F8003E9A071EBFD5F88C
:102DB000003E23F00303C5F8003ED5F8043823F0A5
:102DC0000103C5F80438FEF787FD330502D5204618
:102DD000FEF776FDB7040CD5D5F8083813F0060FCA
:102DE000EB6823F470530CBF43F4105343F4A05327
:102DF000EB60300704D56368DB680BB12046984769
:102E0000F10200F1A180B2020BD5D4F89080002726
:102E10004FF00109D4F894309B68F9B28B4280F0EE
:102E2000D280F3061AD5D4F890100A6AC2F30A17B2
:102E300002F00F0302F4F012B2F5802F00F0EC80E4
:102E4000B2F5402F0AD104EB830301F58051DB6812
:102E5000186A00231A469F4240F0D1803003D5F80B
:102E6000185835D5E90303D500212046FFF7AEFEFB
:102E7000AA0303D501212046FFF7A8FE6B0303D563
:102E800002212046FFF7A2FE2F0303D5032120468F
:102E9000FFF79CFEE80203D504212046FFF796FECB
:102EA000A90203D505212046FFF790FE6A0203D54B
:102EB00006212046FFF78AFE2B0203D50721204674
:102EC000FFF784FEEF0103D508212046FFF77EFEC1
:102ED000700340F1C980E90703D500212046FFF7C0
:102EE00009FFAA0703D501212046FFF703FF6B075F
:102EF00003D502212046FFF7FDFE2F0703D503214E
:102F00002046FFF7F7FEEE0603D504212046FFF723
:102F1000F1FEA80603D505212046FFF7EBFE690662
:102F200003D506212046FFF7E5FE2A0603D5072133
:102F30002046FFF7DFFEEB0540F196802046082192
:102F4000BDE8F047FFF7D6BED4F890904FF00008E8
:102F50004FF0010AD4F894309B685FFA88F7BB42BF
:102F6000FFF451AF09EB4713D3F8002902F44022D4
:102F7000B2F5802F24D1D3F80029002A20DAD3F823
:102F8000002942F09042C3F80029D3F80029002A12
:102F9000FBDB3946D4F89000FFF7D6FB22890AFA0A
:102FA00007F322EA0303238104EB8703DB689B68B2
:102FB00013B139462046984739462046FFF780FB33
:102FC00008F10108C6E708EB4112D2F8003B03F410
:102FD0004023B3F5802F10D1D2F8003B002B0CDA40
:102FE000628909FA01F322EA0303638104EB810396
:102FF000DB68DB680BB12046984701370AE713F01E
:10300000030F08BF0A68072B98BF027003F1010382
:103010009CBF120A01301EE704EB830301F58051C7
:10302000DA6890690268D0F808C04068A2EB000E28
:1030300000221046974208D1DB689B699A683A449F
:103040009A605A6817445F6008E712F0030F08BFE0
:103050000868964588BF8CF8000002F1010284BF21
:10306000000A0CF1010CE5E7BDE8F08708B503485C
:10307000FFF788FEBDE80840FFF776BA84350024E4
:1030800008B50348FFF77EFEBDE80840FFF76CBABD
:1030900020360024D0F8903003EB4111D1F8003BEA
:1030A00043F40013C1F8003B70470000D0F89030A3
:1030B00003EB4111D1F8003943F40013C1F8003992
:1030C00070470000D0F8903003EB4111D1F8003B7D
:1030D00023F40013C1F8003B70470000D0F8903093
:1030E00003EB4111D1F8003923F40013C1F8003982
:1030F0007047000030B5039C0172043304FB0325C4
:10310000C361049B03630021059B00604060C160B4
:10311000426102618561046242628162C16243630D
:1031200030BD00000022416A41610161C2608262DB
:10313000C2626FF00101FEF7EFBE00000369426951
:10314000934203D1C2680AB100207047181D70472E
:1031500003691960C2680132C260C269134482699E
:103160000361934224BF436A03610021FEF7C8BE96
:1031700038B504460D46E3683BB16269131D126819
:10318000A3621344E362002038BD237A33B9294691
:103190002046FEF7A5FE0028EDDA38BD6FF00100ED
:1031A000FBE70000C368C269013BC3604369134485
:1031B00082694361934224BF436A4361002383626F
:1031C000036B03B11847704770B52023044683F39F
:1031D0001188866A3EB9FFF7CBFF054618B186F322
:1031E0001188284670BDA36AE26A13F8015BA362E6
:1031F000934202D32046FFF7D5FF002383F31188C3
:10320000EFE700002DE9F84F04460E469046994638
:10321000202787F311880025AA46D4F828B0BBF1EF
:10322000000F09D149462046FFF7A2FF20B18BF3DA
:1032300011882846BDE8F88FA16AE36AA8EB050B60
:103240005B1A9B4528BF9B46BBF1400F1BD93346F9
:1032500001F1400251F8040B43F8040B9142F9D1FB
:10326000A36A40334036A3624035A26AE36A9A42B9
:1032700002D32046FFF796FF8AF311884545D8D23E
:1032800087F31188C9E730465A46FDF78FFDA36AD8
:103290005B445E44A3625D44E7E7000010B5029C16
:1032A0000172043303FB0421C36100238362C36200
:1032B000039B0363049B00604060C4604261026141
:1032C000816104624262436310BD0000026AC26011
:1032D000426A4261026100228262C2626FF00101B1
:1032E000FEF71ABE436902699A4203D1C2680AB165
:1032F00000207047184650F8043B0B6070470000F0
:10330000C368C2690133C36043691344826943617E
:10331000934224BF436A43610021FEF7F1BD0000E0
:1033200038B504460D46E3683BB123691A1DA26215
:10333000E2691344E362002038BD237A33B9294699
:103340002046FEF7CDFD0028EDDA38BD6FF0010014
:10335000FBE7000003691960C268013AC260C269F4
:10336000134482690361934224BF436A03610023CB
:103370008362036B03B118477047000070B52023C8
:1033800004460E4683F31188856A35B91146FFF766
:10339000C7FF10B185F3118870BDA36A1E70A36AC0
:1033A000E26A01339342A36204D3E16920460439FF
:1033B000FFF7D0FF002080F3118870BD2DE9F84F92
:1033C00004460D4691469A464FF0200888F311882E
:1033D0000026B346A76A4FB951462046FFF7A0FF23
:1033E00020B187F311883046BDE8F88FA06AE76AFC
:1033F000A9EB06033F1A9F4228BF1F46402F1BD947
:1034000005F1400355F8042B40F8042B9D42F9D1F7
:10341000A36A4033A3624036A26AE36A9A4204D3A5
:10342000E16920460439FFF795FF8BF311884E457B
:10343000D9D288F31188CDE729463A46FDF7B6FC84
:10344000A36A3B443D44A3623E44E5E70269436905
:103450009A4203D1C3681BB9184670470023FBE7A3
:10346000836A002BF8D0043B9B1AF5D01360C36825
:10347000013BC360C3691A44836902619A4224BF55
:10348000436A0361002383620123E5E700F04AB940
:103490004FF08043002258631A610222DA607047BD
:1034A0004FF080430022DA60704700004FF0804305
:1034B00058637047FEE7000010B5194CFEF716FC84
:1034C000FEF738FD802217492046FEF7BDFC012398
:1034D00044F8180C0374144B144AD96821F4E061C1
:1034E0000904090C0A431249DA60CA6842F0807282
:1034F000CA60104A1049C2F8B01F116841F00101BA
:1035000011601022DA77202283F82220002383F32F
:10351000118862B60948BDE81040FEF7B7BC00BF8D
:10352000442E0024A83E000800ED00E00003FA0548
:10353000F0ED00E0001000E055CEACC5B03E000854
:103540002DE9F84F1F4C4FF00008656904F114078E
:10355000C1464FF08043266A5B6AAA689E1B96426A
:103560001DD34FF0200AAA68236AD5F80CB0134483
:1035700023622B68BB425F60A6EB02066361C5F85D
:103580000C8001D1FFF78CFF89F311882869D84797
:103590008AF311886569AB689E42E4D2D9E7626913
:1035A000BA420CD0916823628E1B9660A8680228EC
:1035B0002CBF1818981CBDE8F84FFFF777BFBDE87F
:1035C000F88F00BF1C2E0024034B59685A68521A0A
:1035D0009042FBD8704700BF001000E04B6843608A
:1035E0008B688360CB68C3600B6943614B6903627E
:1035F0008B6943620B6803607047000008B52C4B71
:103600002C48D3F8882040F2FF710A43C3F8882081
:10361000D3F8882022F4FF6222F00702C3F8882042
:10362000D3F88820D3F8E0200A43C3F8E020D3F889
:1036300008210A43C3F808211F4AD3F8083111466C
:10364000FFF7CCFF1D4802F11C01FFF7C7FF1C4824
:1036500002F13801FFF7C2FF1A4802F15401FFF7E7
:10366000BDFF194802F17001FFF7B8FF174802F1DA
:103670008C01FFF7B3FF164802F1A801FFF7AEFF78
:10368000144802F1C401FFF7A9FF134802F1E00159
:10369000FFF7A4FF114802F1FC01FFF79FFF10485C
:1036A00002F58C71FFF79AFFBDE8084000F014B9ED
:1036B0000044025800000258D03E0008000402589E
:1036C00000080258000C025800100258001402585A
:1036D00000180258001C025800200258002402580A
:1036E0000028025808B500F0C7FAFFF7E5FEBDE86C
:1036F0000840FEF7A7BD0000704700004FF0804370
:1037000010B51A69920708D500241C61202383F3A1
:103710001188FFF715FF84F31188BDE81040FEF70C
:1037200023BF0000134BD3F8E82042F00102C3F896
:10373000E820D3F8102142F00102C3F810210E4A0C
:10374000D3F81031D36B43F00103D3634FF08043C0
:103750002F229A624FF0FF32DA6200229A615A6396
:10376000DA605A6001225A6108211A601C20FDF7B4
:1037700095BC00BF004402580010005CF8B5514BE6
:10378000D3F880204FF0FF32C3F880200024D3F814
:103790008010C3F88040D3F88010D3F88410C3F8A9
:1037A0008420D3F88410C3F88440D3F88410D96FF0
:1037B00041F0FF4141F4FF0141F4DF4141F07F015D
:1037C000D967D96F21F0FF4121F4FF0121F4DF41D6
:1037D00021F07F01D967D96FD3F888106FEA415182
:1037E0006FEA5151C3F88810D3F88810C1F30A0169
:1037F000C3F88810D3F88810D3F89010C3F890203D
:10380000D3F89010C3F89040D3F89010D3F89410E8
:10381000C3F89420D3F89410C3F89440D3F89410CC
:10382000D3F89810C3F89820D3F89810C3F89840AC
:10383000D3F89810D3F88C10C3F88C20D3F88C10E0
:10384000C3F88C40D3F88C10D3F89C10C3F89C209C
:10385000D3F89C20C3F89C40D3F89C3000F0ECF9DE
:10386000194B07229A60194ADA60194A1A6105222F
:103870005A60184A536A43F480335362C2F8844052
:10388000BFF34F8FD2F88030C3F3C904C3F34E3374
:103890005B01A50743F6E07603EA060E28462146BB
:1038A0004EEA00070139C2F874724F1C00F1404023
:1038B000F6D1203B13F1200FEED1BFF34F8FBFF3B2
:1038C0006F8FF8BD0044025890ED00E00000043016
:1038D0001B00080300ED00E05D4B5E4901221A6009
:1038E0005D4B19609A605D4ADA6000221A614FF4FC
:1038F00040429A619A699204FCD51A6842F4807237
:103900001A60574B1A6F12F4407F1FBF4FF480327A
:103910001A6700221A671A6842F001021A60504AB8
:10392000134611684807FCD5002111611A6912F08D
:103930003802FBD1012119604FF0804159605A676C
:10394000484ADA62484A1A611A6842F480321A60B8
:10395000434A134611688903FCD5116841F0800180
:1039600011601A68D205FCD5404A41499A6200228A
:103970005A636FF401701963A1F500310144DA63F1
:1039800099635A643B4A1A643B4ADA621A6842F005
:10399000A8521A60324B1A6802F02852B2F1285F1E
:1039A000F9D148229A614FF48862DA6140221A62A2
:1039B0004FF00052DA644FF4500100221A65596545
:1039C0009A652E4A202111601A6942F003021A6199
:1039D000234B1A6902F03802182AFAD1D3F8DC20F6
:1039E00042F00052C3F8DC20D3F8042142F0005228
:1039F000C3F80421D3F80421D3F8DC2042F080423C
:103A0000C3F8DC20D3F8042142F08042C3F804213B
:103A1000D3F80421D3F8DC2042F00042C3F8DC20C4
:103A2000D3F8042142F00042C3F80421D3F8042162
:103A3000D3F8F42042F00202C3F8F420D3F81C219A
:103A400042F00202C3F81C21D3F81C31704700BFBA
:103A50002004025100C000F000480258020000019A
:103A6000004402580000FF01008890081210400036
:103A70001702030180020101FF07FF01002000522D
:103A8000084A08B5936811680B4003F0010393607E
:103A900023B1054A13680BB150689847BDE8084048
:103AA000FEF762BD80000058D0380024084A08B5EF
:103AB000936811680B4003F00203936023B1054A39
:103AC00093680BB1D0689847BDE80840FEF74CBD3D
:103AD00080000058D0380024084A08B5936811685F
:103AE0000B4003F00403936023B1054A13690BB143
:103AF00050699847BDE80840FEF736BD8000005881
:103B0000D0380024084A08B5936811680B4003F0C8
:103B10000803936023B1054A93690BB1D0699847B4
:103B2000BDE80840FEF720BD80000058D0380024D2
:103B3000084A08B5936811680B4003F010039360BE
:103B400023B1054A136A0BB1506A9847BDE8084093
:103B5000FEF70ABD80000058D0380024174B10B57E
:103B60009C681A68144004F478729A60A30604D51D
:103B7000134A936A0BB1D06A9847600604D5104A7D
:103B8000136B0BB1506B9847210604D50C4A936B0D
:103B90000BB1D06B9847E20504D5094A136C0BB101
:103BA000506C9847A30504D5054A936C0BB1D06CB3
:103BB0009847BDE81040FEF7D7BC00BF8000005812
:103BC000D03800241A4B10B59C681A68144004F4CD
:103BD0007C429A60620504D5164A136D0BB1506D94
:103BE0009847230504D5134A936D0BB1D06D9847C0
:103BF000E00404D50F4A136E0BB1506E9847A10430
:103C000004D50C4A936E0BB1D06E9847620404D56C
:103C1000084A136F0BB1506F9847230404D5054A27
:103C2000936F0BB1D06F9847BDE81040FEF79CBC76
:103C300080000058D0380024062108B50846FDF75A
:103C40002DFA06210720FDF729FA06210820FDF7A5
:103C500025FA06210920FDF721FA06210A20FDF7A1
:103C60001DFA06211720FDF719FA06212820BDE8C4
:103C70000840FDF713BA000008B5FFF77FFD00F01C
:103C80000DF8FDF7B1FBFDF77BFDFDF74DFCFFF7F0
:103C900033FDBDE80840FFF7F9BB000000230449ED
:103CA0001A465A50C8180833802B4260F9D1704721
:103CB000D038002410B501390244904201D10020CF
:103CC00010BD10F8013B11F8014FA342F5D0181BAD
:103CD00010BD0000034611F8012B03F8012B002A48
:103CE000F9D17047121012131211000053544D33C2
:103CF0003248373F3F3F3F3F0000000000000000D8
:103D0000B11300089D130008D9130008C51300085B
:103D1000D1130008BD130008A9130008951300086B
:103D2000E513000800000000A11400088D1400082D
:103D3000C9140008B5140008C1140008AD14000827
:103D400099140008851400082515000800000000DB
:103D50000100000000000000020000000000000060
:103D6000CD1600083917000840004000F432002446
:103D700004330024020000000000000003000000E3
:103D8000000000007D170008000000001000000087
:103D900014330024000000000100000000000000B7
:103DA000843500240101020025424F415244250080
:103DB0002553455249414C25004E75636C656F484B
:103DC00037343300303132333435363738394142C5
:103DD00043444546000000004172647550696C6FB1
:103DE000740025424F415244252D424C00000000F2
:103DF000E52100085120000839160008C9210008F3
:103E000043000000083E000809024300020100C010
:103E1000320904000001020201000524001001051E
:103E20002401000104240202052406000107058282
:103E3000030800FF09040100020A00000007050151
:103E4000024000000705810240000000120000004F
:103E5000543E000812011001020000408304405744
:103E60000002010203010000040309040000000035
:103E7000ED180008CD1B0008791C00084000400028
:103E8000BC360024BC36002401000000CC360024DF
:103E90008000000040010000080000000001000058
:103EA00000040000080000006D61696E0000000061
:103EB000C83E0008D8360024D03800240100000095
:103EC000B53400080000000069646C650000000063
:103ED0000000802A00000000AAAAAAAA0000000090
:103EE000FFFF00000000000000A00A00000000002A
:103EF00000000000AAAAAAAA00000000FFFF00001C
:103F000000000000000000000000000000000000B1
:103F1000AAAAAAAA00000000FFFF000000000000FB
:103F2000000000000000000000000000AAAAAAAAE9
:103F300000000000FFFF0000000000000000000083
:103F40000000020000000000AAAAAAAA00000100C6
:103F5000FFFF00000000000007000000002000003C
:103F600000000000AAAAAAAA00100000FFFF00009B
:103F7000000000070000000000000000000000003A
:103F8000AAAAAAAA00000000FFFF0000000000008B
:103F9000000000000000000000000000AAAAAAAA79
:103FA00000000000FFFF0000000000000000000013
:103FB0000000000000000000AAAAAAAA0000000059
:103FC000FFFF0000000000000000000000000000F3
:103FD00000000000AAAAAAAA00000000FFFF00003B
:103FE00000000000000000000000000000000000D1
:103FF000AAAAAAAA00000000FFFF0000000000001B
:104000000000000000000000FF00000000000000B1
:10401000EC3C00083F000000009600000000080093
:1040200004000000683E00080000000000000000DE
:104030000000000000000000000000000000000080
:00000001FF
